:400000000010002011000000990400009904000010B502F099FE00F047FAC04610B5174C12232360182002F001FEB0221201144B1A60144B144A1A60FE210902134A1160CA
:40004000134A1A6080218900124A1160124A1A600022124B1A604223114A1360114A1360114A1360114A13604022114B1A600132104B1A601123236010BDC04630001040FC
:40008000080301400000014042FF00800003014040FF00800403014041FF0080280003401801014014010140100101400C010140080101400001014010B572B6184A194BED
:4000C0001A60194A194B1A60194A1A4B1A60EE221202194B1A604E22184B1A600132184B1A601832174B1A603E32FF32164B1A602D3AFF3A154B1A604732154B1A60154AD6
:40010000154B1A607022154B1A60154A154B1A600E22154B1A60FFF781FF00F0ADF910BD6666000600000240EE686606000102400000808000020240000302400000044077
:400140001800044000010440080104401801044000020440B66D03000802044000030440806DDB00080304401804044010B5064C2378002B07D1054B002B02D0044800E08E
:4001800000BF0123237010BD68010020000000007C3D0000084B10B5002B03D00749084800E000BF07480368002B00D110BD064B002BFBD09847F9E7000000006C0100204F
:4001C0007C3D0000800000200000000010B5012002F000FC012002F0F1FB012002F0E2FB012002F0D3FB012002F0C4FB10BDC04610B5032000F01AFE0400032002F012FB47
:40020000704B9C4221D0704B1C602300283B132B02D801226D4B1A70132C02D803226B4B1A702300143B132B02D80222674B1A7023003C3B132B02D80422644B1A70503CF5
:40024000142C02D80522614B1A70604B5A78052A00D9A3E093005E4AD3589F4600225D4B1A705A4C0123A370FFF7B0FF002002F099FB2378042B02D10421544A5170022BEA
:4002800000D08EE00222514B5A708AE00123514A13704E4CE370002002F084FB002002F075FB012002F066FB2378012B02D10121464A5170052B02D10522444B5A70424B39
:4002C0001B68312B6DD99800C0180001C01A424B9C46604402F05EFD63E0002002F04AFB3A4B1B78012B02D10121384A5170042B02D10422354B5A70334B1B68312B50D920
:400300009800C0180001C01A334B9C46604402F041FD46E001222F4B1A7000222B4BDA70294B1B68322B07D84F20404258432B4B9C46604402F02EFD002002F033FB0020D7
:4003400002F03CFB012002F045FB204B1B78012B02D101211D4A5170032B22D103221B4B5A701EE0184B1B68322B07D84F20404258431A4B9C46604402F00CFD002002F0A0
:4003800029FB124B1B78012B02D101210F4A5170022B06D102220D4B5A7002E001220B4B5A700C4B1B78012B01D102F045FD094B1B78002B01D102F0CFFC044BD87802F031
:4003C0004BFD10BDFFFF00006802002084000020803D00008401002092F0FFFF6E0F000010B562B600F0BAF888204000134A010000F028F900F0FAFA02F098FA012400E01A
:400400000324022C0DD0032C12D0012CF9D100F00FFF0028F5D100F02FFD00F05FFF0134EFE700F005FF0028EAD002F075FCE8E700F0FAFAFFF7DCFE0124E2E780020020D5
:400440000B4B1B68002803D080221206134301E05B005B08064A1360064B1B68002802D02022134301E020229343024A13607047002002402800034010B580225201044B8B
:400480001A601122034B1A600120FFF7D9FF10BD94020B40C0020B4010B503F031FC03680C2B00D1FEE7FEE770B50F4E0F4D13E029686B68AC68002202E001C901C30432EA
:4004C000A242FAD1E868002202E0002102C304328242FAD11035013E002EE9D103F016FCFFF77EFFFEE7C046010000008040000010B500230AE0032B03D89A000849505850
:4005000000E008489900084A885001331F2BF2D9FFF7D2FD80229205044B1A6010BDC04600000000990400000000002008ED00E010B5072002F0A4FA10BDC04610B500F04F
:400540001DF810BD10B5044A1368802109060B431360FFF7EDFF10BD0000084010B5064B1B78002B04D1FFF7E9FF0122024B1A70FFF7E8FF10BDC0468801002010B5802262
:4005800052001B4B1A601B4A1B4B1A601B4B1C4A136000241B4A14601B491C4A11601C4A13601C4B1C60072002F074FA0321072002F098FA1849072002F082FA174B1C6067
:4005C000174B1C605222FF32164B1A60164B1C60164B1C60164B1C60503AFF3A154B1A70154B1C70154B1C80154B1C8010BDC04600000840000800406000084007010080E2
:4006000000030840040308401000FE0010030840000208400402084075060000C80E0840880E0840480F0840080F0840C80F0840880F084070020020740200206E020020F4
:400640006C02002070B506000D00141E0BD0072002F020FA044B1C60044B1E80044B1D80072002F00DFA70BD780200207C0200207202002070B5B44B1B68002B00D0984736
:40068000B24B1C88B24B1D68B24B1E680223FF331D4239D0B04A13685B005B081360AF4A137820218B431370117810230B43DBB21370AB4B1B68DB060CD4A44B1A88A94B40
:4006C0001B889A420CD0A54A117808230B43DBB2137005E0A14A117802230B43DBB21370A14A1168A14B0B4013600023A04A13609B4A136002229F4B1A70974A1368802147
:4007000009060B4313601BE1F30602D500229A4B1A600A23334200D1A3E0984B1B685B0769D5974B1A68934B1B78012B04D0002B22D0022B16D057E0924B1B88002B0DD0DC
:400740000121914B1960914B1B681B19D2B21A7001348C4A1388013B138048E002228A4B1A6044E00121884B1960D2B2854B1A800022804B1A703AE0824B1B881B021A4356
:40078000834B1B889A422BD201217F4B1960814B1B889A4202D29B1A9BB200E0002379490B80072B03D80121724B197014E0082B09D16D490B68A020000203430B600021E6
:4007C0006B4B196008E068490B688020800103430B600821664B1960624B1A80140006E00222694B1A6002E0002002F067F90422694B1A6035E05C4B1B689B0431D5B307C0
:400800000DD5664B1B681F211940574A1068574B03401360012014E00821012011E0594B1988083989B219800829F5D8002008E0564B1B681B19524A1268D2B21A70013437
:4008400001390029F4D1002808D1474A1368802109020B4313600022454B1A600C224E4B1A60B3074BD5EB0615D50023404A13603B4A13603B4B1B889C4201D1022300E0BE
:400880000A232B40354A11780B4320218B4313700222384B1A706B062FD5304A117820230B43DBB213702F4B1B881C003C4A1268D20612D5364A1288D31A324A1380394BDC
:4008C0001A68802149020A431A601968364A0A401A601022224B1A6002E00422244B1A600122324B1A603249194B196031490868102303430B60244B1A60154B1D60154B8E
:400900001B685B071CD51F4B1B88002B0CD01F4B1B681B191B78DBB2274A13600134194A1388013B138002E0FF22234B1A60234B1B681F221340082BE5D10F3A204B1A601F
:40094000024B1C8070BDC0468C0100206E020020400F0840000E08400000084074020020880F08406C02002060000840FF5FFFFFC80F084070020020880E0840CC0F084030
:4009800040030840900100206C000840780200207C02002072020020C00F0840080308406400084004020840FFFFFEFF800E0840FF0F0000480F08404002084008020840BD
:4009C000800F084010B5084B1B78002B06D100F0E7F900F047FA0122034B1A7000F058F800F064FE10BDC0469201002010B5FFF7E9FF041E02D100F0CDFD0400002C02D10A
:400A000000F06CFC0400002C03D100F011FC0028FBD100F0C1FA00F007FB002C01D101F0E9FE200010BDC04670B5174E0024002526E06B0904339B00144A9B581F222A40E8
:400A4000D340DB071AD5F37E012B02D0022B09D011E0300000F086F804003100280000F069F90BE0300000F061F804003100280000F0C8F802E0002002F020F828360135CE
:400A8000032DD6D9200070BDA03D00008002002070B5002309E01D491A1D92008818002444600120404250500133002BF3D0184C042327E06668A27E144B5B19002119765B
:400AC000012A04D0002A1BD0032A08D918E02069002815D0F179228B03F047F910E02369002B01D0F2791A706168002306E01A1D52008A1801204042D0800133002BF6D07A
:400B000028342B005D1E002BD4D170BD80020020A03D000030B50B884A889C1A0025CD800079844200DDCC8030BDC046F0B583B08468038B4568877E002201920BE03A008C
:400B40002100280000F086FA019021002800FFF7E1FF0A3433005E1E002BF0D1019803B0F0BDC046F0B583B0070084684568837E01930026002300930BE0019A210028007C
:400B800000F068FA009021002800FFF7C3FF0A3401363B8B9E42F0D3009803B0F0BDC046F0B50A8B8D684F680B69012125E00C00044003D17E88BA79B21802E07A88BE79B3
:400BC000921BEE88B24201D3002200E00A00A24202D01E78013E1E70A24202D01C78002C07D188431043002A01D1FA7900E001221A7049000A3501336246541EA446002A93
:400C0000D5D1F0BD70B504008A7E134B1B181D7E012A04D12800FFF7C3FF050002E0002001F04CFF0C4B1B191D7663091F2214401E3AA240002D07D104339B000649CB187F
:400C400059689143596006E004339B000249CB1859680A435A6070BD80020020F0B5474680B482B084460F000B8B8A684D6809698846002803D16888A979401802E0698882
:400C8000A879081A0024012109E0D388984201D3002300E00B001C430A32490033005E1E002BF2D1002C0CD043461B78002B02D0013B4246137043461B78002B04D06446FD
:400CC00002E0EB7942461370002C0AD06B88AA799A1A3E8B3100B86801F0AAFC002802D121E000201FE0BB7E022B1CD1396A0023320001A801F008FD00220AE0530002A913
:400D00008C466344043B1988131D5B00EB18D98001329042F2D806E0031D5B00EB1801225242DA8001300028F6D0200002B004BC9046F0BD70B504008A7E184B1B181D7E99
:400D4000012A04D0002A0CD0032A05D909E02800FFF726FF050007E02800FFF77FFF050002E0002001F0AAFE0C4B1B191D7663091F2214401E3AA240002D07D104339B00DF
:400D80000649CB1859689143596006E004339B000249CB1859680A435A6070BD8002002070B51D4C882252000021200002F0DDFF1A4B238090231B016380194BA380082331
:400DC000A3830126A677E677164D20002030290028313A2202F0C0FF80235B00E6502000AA3029006431562202F0B6FF0E490C00083404230CE0A268238B04E00B78537229
:400E000001310A320300581E002BF7D128342B005D1E002BEFD170BD8002002084330000B80B0000183E0000983D0000032811D882001218D300094AD31822331B78023B81
:400E4000DBB2012B08D883001818C300D318DB68D88902E0024800E001487047983D0000FFFF00000023024AD380024A1360704780020020A401002070B500250026414B5A
:400E80001B68032B06D102F004F801223E4BDA8002F003F83C4BDC88E4B2062C23D8A3003A4AD3589F460122364B1A6001261AE00022344B1A60012615E0FFF797FD0022C2
:400EC000304B1A60012501260DE002222D4B1A60012608E000222B4B1A60012603E00322284B1A600026002E0FD001F0D2FF264BDB88DBB29C4205D1234AD188244B0B43E3
:400F00009BB2D38001F0C9FF00261E4B1B68012BB5D0022B33D11C4A0733FF33D35CDBB20A21FF31525CD2B2032B28D89800C018C10018484118098B8A4220D212490889F3
:400F400080B285246400095B89B2884217D09900CB18D9000F4B59188C6893009A185300E41801F096FF084B1A8992B2852149005A52228892B202315A5201F08EFF28006C
:400F800070BDC046A401002080020020084000000080FFFFA03D00007047C046FF231940062902D08318002119715300195AC31859808218002313727047C04670B50600D1
:400FC0000D00012305E0220029003000FFF7E6FF23005C1E002BF6D170BDC04670B5074D86003218D4002C19A0688A0051184A008018A17EFFF7E2FF70BDC046A03D00007E
:4010000070B5050082001218D300064AD3181B8B04E021002800FFF7E1FF23005C1E002BF7D170BDA03D000010B5042303E02000FFF7E6FF23005C1E002BF8D110BDC0465B
:401040009840504380235B009A1A51434018000A7047C046F0B5474680B482B007000E00019201233EE06300985BF3185988884205D3431A321900251572012201E00B1ABD
:401080000022002A11D17D79AB420ED933191B7A3A7A934205D3220001993000FFF77EFF1FE03219013313721BE03D79AB4204D97D79AB4215D2002A13D1FF23019A134031
:4010C000062B0ED00902331998461B79194308230122FFF7B5FF020A6300F3185A804346187123005C1E002BBDD1002002B004BC9046F0BD70B504000D009F2808D91B4BAF
:40110000994205D91A49280002F00AFD002921D09F2C09D9FF235B009D4205D91549280002F0FEFC002917D09F2C07D97E2D05D97F21280002F0F4FC00290FD09F2C0FD956
:401140003E2D0FD93F21280002F0EAFC00290BD000200AE0042008E0032006E0022004E0002002E0002000E0012070BDFE030000FF030000FF01000010B54B1EDBB2032B57
:4011800001D8102300E00023002911D0002B11D0642253430100180002F03CFC002301E0013340000928FBD90A2804D9013B02E0002300E00023D8B210BDC04610B5064A69
:4011C0001368F0218B431360044A1368EF398B43136000F043FD10BD00040240A8020B4010B5064B1968064A0A401A601968054A0A401A6001F0CAF910BDC04600040240AC
:40120000FFF0FFFFFF0FFFFF70B50D000C8801F005FA06002100FFF76DFF040001003000FFF7AAFF0001C0B22043287370BDC046024BDB68802018407047C0468002002017
:4012400010B5164BDB68DB030DD403280DD8430904339B00114A9B581F220240D340DB0705D4012404E0112402E0012400E00024002C11D182001218D300094AD318DB7E0C
:40128000012B04D0022B05D101F092F904E000F0F7FC01E001246442200010BD80020020A03D000010B50B4BDB68DB030DD40A4B1B78012B05D0022B09D101F0A5F8002015
:4012C00007E000F057FC002003E0112001E00120404210BD80020020A801002010B50F4BDB681B0618D400240120404211E02000FFF7A6FF00280BD1022C03D80122084B6F
:401300005A7002E00022064B5A70FFF7CBFF04E00134032CEBD900E0112010BD80020020A8010020F8B5160083001818C300364A9C58CB00591A8B00E418002561E001F0E6
:40134000A8FD21680B68277E0F22BA4093430B6061680B68A77E0722BA4093430B6001F09CFD052E4BD8B300284AD3589F4601F090FD62681168A77E0623BB400B43136016
:40138000A1680B68677E0122BA4093430B6001F084FD34E001F07DFDA1680B68677E0122BA4093430B6001F078FD28E0200000F0C7FB24E001F06DFD22681168277E042350
:4013C000BB400B43136062681168A77E0623BB400B43136001F061FD11E001F05AFD22681168277E0623BB400B43136061680B68A77E0722BA4093430B6001F04EFD1C347E
:401400000135002D9BD0F8BDA03D00002440000010B50400124B1B7883421FD0012B02D1FFF7CCFE03E0022B01D1FFF7D9FE012C05D100F007FA0122094B1A700EE0022CFC
:4014400005D100F069FE0222054B1A7006E0042C04D0032C02D00022014B1A7010BDC046A801002030B500200D4B16E019680A681C69A2430A605C6822689D7E0721A9402E
:401480008A4311000622AA400A43226099680A685C69A2430A601C3301300A28E6D930BDD43E000010B51B4A93780133DBB293709078C0B2FFF7C4FE041E09D1154B9B78DC
:4014C000032B02D10022134B5A70FFF7EBFE1EE0104B9B78032B11D10F4B1A8901321A81DA6880218A43DA60DA681202120ADA60DA6804061443DC60002408E0064AD3686F
:401500001B021B0AD360D16803060B43D360002CC9D110BDA80100208002002010B501F08DFA10BD074A084B1A6001380002074B1860054B1B68002BFBDB054A024B1A605E
:401540007047C04640000040000001400003014040FF008070B50400032801D8002500E00125002D12D1A2001219D300084AD318DE7E022E03D12821200000F0BBFE012E04
:4015800004D15521200000F057FC0500280070BDA03D000070B50024002504E02000FFF7D9FF05430134032CF8D9280070BDC04670B500251EE0AA005219D3000F4AD318BA
:4015C000DB7E012B15D1AB005B19DA000B4BD658002406E0E3001B1B9800301800F01EFB0134AA005219D300044AD3181B7E9C42F0D30135032DDED970BDC046A03D00003A
:4016000083001818C300024AD3185B6858897047A03D00000203121A01238B40013B9A4205D90202101A834203D3052002E0062000E00020C0B2704770B50E00FFF7E0FF88
:4016400005003188002200F0ADF901002800FFF751FD041E04D168003188FFF7DBFF040021002800FFF788FD0001C0B22043307370BDC04610B5002413E0A2001219D300AF
:40168000094AD3185968DB7E012B02D0022B04D006E02000FFF7D0FF02E02000FFF7B4FD0134032CE9D910BDA03D000010B5FFF7E1FFFFF7D7FE0020FFF7AAFE002010BD7E
:4016C00070B501F0E6FB134A1168134B0B40136001F0E3FB01F0DDFB104A13680E218B43136001F0DAFB01F0D4FB0D4C23680D4D2B40DB2212011343236001F0CEFB012031
:4017000001F000FB01F0C5FB23681D40256001F0C4FB70BD000402400F00FFFF000404400804044007F0FFFF01390843014B18607047C04600020B4010B50F4B1B6870225B
:4017400093431C000D4B997F0D4802F063F90D4B984204D820232343074A13600BE0084B984204D830232343034A136003E040232343014A136010BD8C00002080020020F7
:4017800000366E01001BB700034A044B1A60C1225204034B1A60704700008301C0010B40C4010B40074B1A687F210A40064802431A60064A13680B40802109040B431360F4
:4017C0007047C046C0010B4000008301C4010B40064A136806490B431360064A064B1A60C1225204054B1A607047C046A8020B400100001000008301C0010B40C4010B4030
:4018000070B50E001500038801249C40013CA3001B195800642102F0FDF8013083199C4200D22300B04201D8301A00E00020A84203D8AB4203D2062002E0062000E0002092
:4018400070BDC04670B5FFF7B3FEFFF739FFC0221203274B1A60274B1968274E314319600024264A1460264A1460264A1460264A1460264A1460264A1460264A1460264D30
:401880002C60264A1460264A1168F0208143903801431160234A1168802040010143116080214900204A11601A6832431A6080235B041E4A13601E491E4A11601E4A1460D3
:4018C0002B60FFF761FF1D4B987FFFF72BFEFFF733FF1B4B1B681B4A13431B4A136001221A4B1A601A4B1C6009321A4B1A6070BD04020B40A8020B4001000010F4000B4005
:40190000B4020B40C0020B4020030B4084010B4088020B4080020B4084020B4080010B400004024094020B40A0020B40A4020B404112000088010B4090020B408002002071
:401940008C0000200010008000000B4000030B40F0010B4010030B4070B5050001F099FA0C490B687F26B3430B4A14782D196A7A13430B6001F091FA01F08BFA07490B6866
:40198000B343074A12681419627A13430B6001F084FA70BDC0010B403C400000C4010B409003002010B503001400012088400138002B02D0190002F02DF8053C012C00D844
:4019C0004008002800D1013010BDC04610B50E4B1B78DBB29A00D318DA000C4B9A18536859891B7B18045A1F012A02D8802292041043053BDBB2012B02D8490800D101317D
:401A0000FFF792FE10BDC046AA010020A03D000010B50300408919881A7BFFF7C3FF0004000C014B186010BD14030B4010B50A2001F030F801222D4B1A6000232C490B6003
:401A40002C490B602C490B6006202C490860FA302B4908602B490A60832149002A4A11602A4A136003222A4B1A60E123DB0100E0013B254A1268520701D4002BF8D1002BC0
:401A800002D10822224B1A60832252001E4B1A600A2001F009F80A2000F0F2FF0023184A1360144A1360144A1360144A13605021144A11604F390E4A11600C4A1360154A1D
:401AC0001368802149040B43136002220F4B1A60E123DB0100E0013B0F4A1268520701D0002BF8D10D4A0A4B1A6010BD80010B408C010B40B0020B40B4020B4088020B406D
:401B000080020B40F0010B40F0000B40F8000B4040030B4000020B4000000B400103000010B5054AD36805490B43D360172001F0E9F8FFF77BFF10BD80020020800001006D
:401B400070B50400857E067E01F0A3F923681B680F22B24093431A000423B3401343666832680721A9408A4332602268136001F094F970BD70B5194E3378DBB2184D9A0054
:401B8000D318DA00AA185068164C002323703378DBB29A00D318DA00AA1891682378DBB29A00D3185A008A180F4B1A60FFF7D4FE3378DBB29A00D318DA0050592278D2B2D9
:401BC000D3009A1A9300C018084B1860FFF7B8FF074800F033FFFFF7A3FF70BDAA010020A03D0000B00100209003002094030020E12F000010B583001818C300054A9858D8
:401C0000CB00591A8B00C018034B1860FFF798FF10BDC046A03D00009403002070B50400007EA57E21680B680F22824093430B6001F02FF961680B680722AA4093431A00F7
:401C40000623AB4013430B6001F027F9A1680B68607E0122824093430B6070BD10B5064B1B78012B06D1054B1868FFF7D7FF0022014B1A7010BDC046B10100209403002035
:401C800070B5124C82001218D300E3185D68C0B20F4E30700120FFF7BBFBFFF7DFFF3378DBB29A00D318DA0012590A4B1A600A4BDA687F218A43DA603178DA680A43DA60D1
:401CC0002800FFF7A5FEFFF781FE70BDA03D0000AA010020940300208002002070B582001218D300134AD3185D68C9B2124C217099682378DBB29A00D3185A008A180F4B61
:401D00001A60FFF7BDFF2800FFF726FE2378DBB20B49DA00D31A98000B689C4660440860FFF70EFF0122074B1A70074800F086FE70BDC046A03D0000B001002090030020A0
:401D400094030020B1010020B52F0000F0B5474680B482B007000E00904630490B78DBB29A00D318DA002E4B9A1853680193002333700878C0B22B4B1978C9B2FFF7AEFF34
:401D8000FFF710FD00248025BC4202D23378AB4333706D0833782B4333700198FFF7DCFDFFF7BEFEE123DB0100E0013B1E4AD268120601D5002BF8D11C4B1B681C88002DC3
:401DC000E2D1164B1B78DBB29A00D318DA00144BD058144B1A78D2B2D3009A1A9300C018134B1860FFF71AFF0022124B1A70FFF7EFFC220039000198FFF702FD43461A788F
:401E000033789A4201D242461370084B1B6832785A7202B004BC9046F0BDC046AA010020A03D0000B0010020800200209003002094030020B1010020F0B54F4680B484B0FD
:401E40000400894682001218D300394AD3185F68012003AB18703B88984001384843642101F0D8FD0190E2B2324B1A70324800F0E5FD3E0009360022304B1A7000250AE0AF
:401E800003AA31000198FFF761FF05432B4A13780133DBB21370A2001219D300244AD3181A7F264B1B78DBB29A42E9D803AB1B7801335B087B720022204B1A7024E0A20087
:401EC0001219D3001A4AD3189E681C4B1B78DBB29A00D3185A00B618194B1E60737A787A83420AD31B1AD8B270724B4658436330642101F08FFD707201E0002373720F4A72
:401F000013780133DBB21370A2001219D300084AD3181A7F094B1B78DBB29A42CFD80022064B1A70280004B004BC9146F0BDC046A03D0000AA010020B52F0000B0010020E5
:401F40009003002043890288981E504380B2704710B5344B1A68344B1B78D3185B7A334A1343334A13600022324B5A80324A334B1A600122324B1A601123324A1360802100
:401F80004904314A1160314A13600622304B1A60304A314B1A60314A314B1A60314A324B1A60F0235B0000E0013B2F4A1268D20701D5002BF8D12C4B1B68DB0703D5C222D2
:401FC0009200294B1A60294BD97F294801F022FD284B984204D9264B984203D8302302E0202300E04023244A1343144A1360234A234B1A60002312490B6012490B60124915
:402000000B6023201149086011490B6012490B6013490B60832149001A4B1960124B1A6010BDC046900300203C400000800E4301C0010B40B40100202010048000000B4088
:4020400080010B4080020B4084020B40C0020B4088020B4001010100B0020B4010100000B4020B400303000040030B408002002000366E01001BB70000100C8001030000A6
:402080008C010B40F0000B4010B50A2000F002FD83225200154B1A60154B1B689BB2154A5380154B1B689BB25188CB189BB25380518889B213889BB2994202D913889BB256
:4020C00053800E4B1B6898470D4BDB681B0609D40C4A0D4B1A60C02292000C4B1A600C4A0C4B1A600A2000F0CBFC10BDF0000B40D0000B40B4010020D4000B40900000207D
:40210000800200202010048000000B408C010B40800E4301C0010B4010B5832252004A4B1A600024494B1C60053AFF3A484B1A60484B1C60484B1C60484A494B1A60C02224
:402140009200484B1A60484A484B1A60484B1C60484A494B1A605022484B1A60484B1C60484B1C60484B1C60484B1C60484B1C6000F08FFE474A1168474B0B408021490159
:402180000B43136000F089FE3222444B1A6080225204434B1A6000F07CFE424A1168424B0B40802149050B43136000F076FE3F4B1C603F4B1C6023223E4B1A60223A3E4BF6
:4021C0001A6003323D4B1A603D4B1C603D4B1C60C22292003C4B1A603C4A3D4B1A60FFF76FFA00F056FE3B4C22683B4B1340236000F053FE00F04DFE2268384B13402360B8
:4022000000F04BFE00F045FE354C2268354B1340C022D2001343236000F03FFE00F039FE2268314B1340C022D2011343236000F034FE2E4BD87FFFF775F9FFF713F92C48C0
:40224000FFF76CF910BDC046F0000B40F4000B40F8000B4080010B4084010B40411F000088010B408C010B40800E4301C0010B40C4010B40AA000500F0010B4000020B40A5
:4022800004020B4080020B4084020B4088020B4090020B4094020B40FFEFFFFFA0020B40A4020B40A8020B40EEFFFEEEB0020B40B4020B40C0020B4000030B4010030B404D
:4022C00014030B4020030B4040030B402010048000000B40080404403FFEFFFFFFF1FFFF00040240FFF0FFFFFF0FFFFF8002002089200000F0B54F4680B482B001900E003F
:40230000830084466344DA002B4CA418A36899462A4B4A461A606068FFF714FE284B188018887043642101F075FB0700E37E022B3ED1019B9A009C466244D3001E4AD31897
:402340001A7F5E7F5643002109E01C4A0023106803801368402058720A3313600131B142F3D32024402500E01C000198FEF768FFFEF798FF134BDB681B06FBD40F4B4A46DF
:402380001A6000210EE00D4B1B681A88974202D25A7AAA435A725A7A22435A720A33074A13600131B142EED36308DBB2251EDBD102B004BC9146F0BDA03D00009003002084
:4023C000B40100208002002010B542681168847E0623A3400B43136002681168007E042383400B43136010BD10B541680B68847E0722A24093430B6002681168007E06231D
:4024000083400B43136010BD10B50022124B1A70124B1B68124A996811605A7F114CA2801A7FE2801968A160D300981A80000818E060FFF7C9FFA068FFF7D6FF0A4A0B4B5A
:402440001A600B4AD16880230B43D360172000F059FCFFF77DFD10BDB0010020AC01002090030020B4010020B124000090000020800200200268136801698B4313607047E3
:4024800010B50268136801698B43136041680B68847E0722A24093431A000623A34013430B608268136841698B43136010BDC04610B52F4B19682F4B1B782F4C22886088E4
:4024C0005B00121A5A52E068FFF7D4FF2B4A13780133DBB21370A388013B9BB2A380002B0CD0254BD8681C30D860FFF76DFF204A13680A331360FFF72BFD37E01E4AD38853
:40250000013B9BB2D380002B1DD014009068FFF7B7FFA0681C30A060FFF766FF184B1B685A7FA2801868E0601A7FD3009A1A9300C018E060FFF748FF0D4A13680A33136015
:40254000FFF706FD12E00C4B9868FFF799FF0D4B1B78002B02D0FEF7A5FF07E00A4B1A8901321A81DA6880218A43DA6010BDC046900300203C400000B4010020B0010020CB
:40258000AC010020A90100208002002010B5074B1B8A002B08D0054CE068FFF76BFFA068FFF76EFF0023238210BDC046B401002070B50400C2B2124B1A700220FEF728FF8D
:4025C000FFF7E4FFA3001C19E2000E4BD3180E4A13605D686C892A880C4B1A602800FFF7B1FC0B4B18802B7B013C2405240D1B041C43084B1C60084BD87FFEF793FF70BD5B
:40260000AA010020A03D0000AC01002014030B40B401002000020B408002002083001818C300024AD3185B6858897047A03D0000F0B50024334B1C700400002600230BE00F
:40264000E588954206D9AE4204D22E4E3371012737702E000A3401338B42F1D3294B1B78002B46D14AE0274FBB181B799E00F61874000519ED88AC465600B61875007D192D
:4026800066466E81002B12D18D006D186C000A3C0419E6885500AD186C003C19268101339D00EB185D004519EB88A3811FE04D1EEDB2AB420BD10A3C0419E5885400A418C8
:4026C0006300104CE3181D81C4889C810FE00A3C0419E6885500AD186C000A4D2C19268101339D00EB185D004519EB88A381013200E00022034B1B789A42B4D3014B187815
:40270000F0BDC046C8010020F0B557464646C0B483B082460F000192984600252DE01B4B5B191C79002C07D16A0052195300174AD31800221A810AE0019B013B9C4206D1F3
:402740006A0052195300114AD31800229A816E00721953000D4AD3189A891989501A5B89C9185118784301F0DFF97C43444400197F30000A534698530135044B18788542C6
:40278000CDD303B00CBC90469A46F0BDC801002010B582001218D300144AD3189B7E023BDBB2012B1ED883001818C300D318586800234B720AE01A1D52008218D4880C4A60
:4027C000944202D04A7A01324A720133002BF2D0C3890B8000234B8001338B72023B8B80CB8002E0002000F069F910BDA03D0000FFFF000010B50948002282235B00C2508E
:40280000074B5A729A721A72013A1A805A809A80DA80AA3001F0B8F810BDC04680020020D801002070B5040003282BD11B4D2900FFF7AEFF2B7A002B0DD0012B1DD1174B29
:402840005B7A002B20D10022144B1A72144801F09BF8002019E0114B587A9B7A984204D901220E4B1A72FE200FE082235B000D4AD1580A4A00F0FCFA07E00122074B1A72B0
:40288000FE2002E0FF2000E0FE20A3001C19E300054AD3185B68587370BDC046D80100202A03002080020020A03D0000154A13685B005B081360F8214901134B1960134BDD
:4028C00013600022124B1A60124B1349196059609960D9601961114858619961D961802119625A629A62DA621A631A3959639963DA630B4B1A600821FF310A4B19600A4B6E
:402900001A60704700000540E40100205F1F0000100005402000054011111100090B0900C0000540C4000540F000054010B50E4B1B79002B05D1FFF7B9FF01220A4B1A71ED
:402940000BE00A4B1B68002B07DB08490A68084B1340054A126813430B60044A1368802109060B43136010BDE401002000000540FFE0FFFD04490A68D2B210239A43000114
:4029800018401043086070470002044004490A68D2B208239A43C00018401043086070470002044004490A68D2B204239A43800018401043086070470002044004490A6856
:4029C000D2B202239A434000184010430860704700020440044A1368DBB201218B430840184310607047C04600020440014B98667047C0460000002010B5040000F049FA82
:402A0000044A1168044B0B40A4051C43146000F044FA10BD08E400E0FFFF3FFF8022D200014B1A607047C04600E100E08022D200014B1A607047C04680E100E010B50400FD
:402A4000FFF7F4FF2000FFF7D1FF0320FFF7D4FFFFF7E4FF10BDC046024A1168024B0B401360704700000740FFFFFFBF034B18688023DB05184000D00120704700000740CD
:402A80001F2318401E3B8340014A13607047C04600E100E01F2318401E3B8340014A13607047C04680E100E01F2318401E3B8340014A13607047C04680E200E001BE7047C9
:402AC00070B504000D000F2802D90020FFF7F6FF1034A40080239B059C4664442068256070BDC04670B504000E00032902D90020FFF7E4FF0F2C02D90020FFF7DFFF032525
:402B00002540ED00063500F0C4F9A408A400074B9C46644421680323AB4099430B003100A9401943216000F0B8F970BD00E400E010B5040006E0084B586800F0A1F9074B87
:402B40009C46644480231B029C42F4D8024B9868604300F095F910BD940000200080FFFF30B583B000F0E6F8002849D000F091F90400244B196889001C2319401831224B88
:402B80001B689B0803221340D940204B1A68204B1340204A4A438020C00184466244D20B013A5205520D1343A02252031A431000192902D8184A13430CE0184BCB181B78AA
:402BC0001A39174A525C9A18FF2A00D9FF229205030013430D4A1360124D2B680193302000F022FA104A13688021C9050B4313601420FFF79DFF019B2B60200000F04DF9BA
:402C000003B030BD080F0340280003400800074000F800C040420F000000D43FCDF1FF0F404000003000104000000740F0B583B0040018280BD01C2809D0202807D02428F2
:402C400005D0282803D02C2801D0302849D100F020F90190FFF70AFF002803D0FFF7FCFE012600E00026214A136807218B4313601F4BE3181B78DBB21E4A13601E4A136882
:402C80008B4313601D4803687F22934319001C4BE3181B7813400B430360322000F0F0F8182C16D9114F3B680725AB431A0023001C3B9B082B4013433B60322000F0E0F853
:402CC0003A68AA432300183B9B082C001C4014433C60012E01D1FFF743FF019800F0DDF802E00020FFF7EAFE03B0F0BD080F0340CDF1FF0F0C0F0340100F0340180F03408A
:402D0000B4F1FF0F10B5034B1B7B584300F0B8F810BDC0469400002010B500F0BAF8044A136804218B43136030BF00F0B6F810BD10ED00E0034B1B68002B01DA012000E0D0
:402D40000020704700000740014A024B1A6070476588EDAC3800034010B500F09AF8044A136808218B43136000F097F810BDC046000006400004000C014B18607047C046C8
:402D8000C80106400004000C014B18607047C046D40106400004000C014B18607047C046CC01064070B504000D0000F072F8AC40024B1C6000F071F870BDC0460800064095
:402DC00010B500F066F8064A116808230B43136000F063F818210820FFF7E4FF10BDC04600000640014B18607047C046F801064010B50E4C8023DB0423602368236000205B
:402E0000FFF7B8FF236823600C22094B1A600120FFF7E8FF3122074B1A60FA200001FFF7B1FFFA20C000FFF7B5FF10BDC0010640E4010640E801064010B5064B1B78002B77
:402E400004D1FFF7D5FF0122024B1A70FFF7B8FF10BDC046E901002004490A687F231A40C301D8B2104308607047C0460003044010B5C0B200F01AFD10BDC0460000000056
:402E80000230800803D001300238FCD1C046C0467047EFF3108072B6704780F310887047104B1B78DBB29A00D318DA000E4B9A1853680E4A11680A04120C18880123834053
:402EC000013B9A4206D20A4B1A680A4B1B785B00D15205E0064A1168064A127852008B527047C046AA010020A03D0000D0000B40900300203C40000070B5274A1378DBB291
:402F0000264C9900CB18D900611848681378DBB29A00D318DA00A218127E013A204B1B78DBB29A4220D91E4C23780133DBB22370194D2B78DBB29A00D318DA00174B9A18E3
:402F400091682378DBB29A00D3185A008A18154B1A60FEF701FD2878C0B22178C9B2FEF749FEFEF763FD16E000220D4B1A700E4AD1680E4B0B40D3600D4B1B78012B02D1DF
:402F8000FEF790FA07E0084BDA6880218A43DA601A8901321A8170BDAA010020A03D0000B00100209003002080020020FFFFFEFFA901002010B583225200064B1A60FFF7C0
:402FC0006FFF054B1A8901321A81D968034A0A40DA6010BDF0000B40800200207FFFFEFF10B50D4B1B78DBB29A00D318DA000B4BD4580B4B1A78D2B2D1008A1A9300E418DD
:4030000083225200074B1A60FFF74AFF2000FEF705FEFFF771FF10BDAA010020A03D0000B0010020F0000B4070B50400FFF731FF0500102C05D8104A136803218B431360E8
:4030400016E0202C07D80C490B6803229343023A13430B600CE0302C07D807490B6803229343013A13430B6002E00020FFF726FD2800FFF712FF70BD300010400023034A27
:403080001370034A1360034A13807047C6030020EC010020FA030020224B1A004D321278824209D81A004E321278904204D81A004C321278D2062CD51A004F32127890422A
:4030C00009D31A0050321278904204D81A004C32127892061DD51A0051321278904209D31A0052321278904204D81A004C32127852060ED51A0053321278904210D31A0074
:403100005432127890420BD84C331B785BB2002B06DB054B1868002802D00123037000207047C046A8000020B0030020074B1A00D9895B8ACB1806495B100B80118A938A33
:40314000044ACB185B1013807047C046EC010020D0030020A2030020064B1968002908D0054B1B68002B04D0044AD0890880128A1A807047C0030020F4030020EC010020D6
:40318000074B1968002909D0064B1A68002A05D0054B588A0E330880DB8813807047C046B4030020DC030020EC010020084B1A68002A0BD0074B1B68002B07D012788242D8
:4031C00001D0012201E01A7801321A707047C046B8030020B0030020F0B5B94B85B01B680700039100921E1E00D01E78B54B1B680193002B01D01B780193B34B00251A7821
:40320000012A03D1B14BDD691B68ED1A012F59D1AE490131CB7F002B29D1AD4BE8B21C0048342488A0421ED8012A1CD1323302931C78A84AA84B12881B88D21AD317D2189B
:403240005A40A2420FDA029BA44C1A78A44B24881B881B1BDC171B196340934203DAA14BCF77188003E00322984B0133DA77974B0133DB7F012B1DD1954A974813003333DD
:403280001978994B00881B881B1AD8171B1843408B420BDC954B91491B88098834325B1AD91712785B184B40934203DD0222874B0133DA77854B24240133DB7F022B1ED0AE
:4032C00000241CE0002F0ED1804C631CDB7F023B012B05D8FFF7D2FE7E4B1F80804B1F80631C00240AE0022FEAD10024FFF7C6FE784B1C807A4B1C80744B0133DC777C4BF9
:403300001C70002C07D02000FFF750FF794B1B68002B00D01C70002F05D0002E00D027E1694B1B789EE0744B1B68002B02D01B78002B05D1714B1B68002B01D001221A7041
:40334000012E00D080E0624B00991A000832D28F002491422AD99A1DD28F914226D219003331614A08785C4912880988891ACC1709196140814200DD9BE034335B4918789F
:40338000564B09881B885B1ADC171B196340834200DD8EE04C480378002B04D1584C2468002C00D0B0E000240133037046490B780800022B45D1464B1A004A32128895425E
:4033C00002D2FFF75BFE3FE01A0048321288954217D2404A444F12883F883233D21BD7171C78D2197A40A2420BDA1A783F4C3C4B24881B881B1BDC171B196340934200DA3B
:403400009DE03F4B1B68002B1ED01B78002B1BD02C4B1B68002B02D01B78002B14D101230370314B20241A882A4B1A802F4B1A882B4B1A80254B039A1A600022294B1A80BB
:4034400096E0002C00D093E0019B1B0603D4022E19D0012E12D00024A64200D088E03400194B1B78012B00D082E0194B48331B889D4200D87CE0FFF701FE79E0019B3340EA
:40348000DCB2002C74D00E4B1B68191E00D019781C4B1B681A1E00D01A780D4B009D181DC08F0024854263D90233DB8F9D424ED35EE00024044B1C700A4B1C8076E7C04646
:4034C000F0030020E4030020C6030020EC010020A8000020E8030020FC030020C4030020AC030020FA030020BC0300209E030020E0030020B8030020EC030020B003002097
:40350000C8030020A40300202478002C00D14AE7194C2468002C03D02478002C00D042E7164B20241A80164B1980164BDA691A600022154B1A80154B01321A7036E7124B54
:40354000104A1D80002322240B70136010E00D4B0233DB7F002B0BD1012902D1002A04D006E0022901D1002A02D0FFF787FD4024200005B0F0BDC046E4030020E8030020CD
:40358000AC030020EC010020FA030020C603002010B50400FFF780FD1349144B84421AD0283C012C17D8124A1278FF2A13D052001032D0B21A79824208D1DA1CD27F0C680F
:4035C0000132D2B2002C06D0227004E00A68002A01D0012414700A68111E00D011780333D977FFF759FD10BDB0030020EC010020CE030020F7B5944F06003B680C00019245
:40360000002B00D115E11B78002811D1002B00D119E18E4A8E49536AA34201D2E31A01E0DB431B190B80D369E41A019B1C600AE1002B07D1854B5C62864B1B68002B01D008
:4036400001221A70844D2B68002B02D01A78002A23D1824AD18E824A1268A21A8A421CD3002B01D001221A70784BDA89DC617D4B1A807D4B5A887D4B1A80FFF76DFD022E9A
:4036800000D0D9E0784B9A88794B1A80764BDA88784B1A80FFF774FD58E0012E53D16B4E019A736AE31A13603B68734F002B02D01B78002B15D1F2896A4B1A80328A6B4BE9
:4036C0001A803B68002B01D001221A702B68002B01D001221A70624BF4611C60FFF73CFD18E0022B16D13B68002B01D000221A702B68002B01D000221A70594B1C605F4B9F
:403700001A68002A06D0012113780B4200D080210B4313703B68002B02D01A78002A0BD12A68002A08D01278002A05D0002B01D001221A70FFF710FDF289514B1A80328A5D
:40374000504B1A807FE0022E00D07CE03B683F4E002B0ED01B78012B24D80AD1474B1A68002A06D0022113780B4200D080210B4313700022B31CDA772B68934200D01A7035
:40378000374BF189374A1C601180318A374A394B1180718A364A1180B28A1A80FFF7DCFCFFF7EEFCB31CDB7F002B33D12B68002B30D01B78002B2DD0284B31001800294A9E
:4037C000F58912883330521BD517047852190E316A40A24233DC254A4D8812883433521BD5171C7852196A40A24228DC204A8C8812880078121BD4171219624082421EDCD0
:403800001A781C4BC9881B885B1AD9175B184B40934214DCF1891A4A1B4B1180318A194A1180718A194A1180B28A1A80FFF77EFC09E0002807D0FDE6012E04D12FE70122B2
:40384000B31CDA77E6E7F7BDF0030020EC010020CC030020B0030020A4030020A8000020D4030020FC030020FA010020C4030020A0030020BE030020C8030020E403002088
:40388000BC0300209E030020D2030020D8030020054B1B681A1E00D01A782F23904200D8203318007047C046F00300200023F0B52E4C87B0059323002D4E733333602300C9
:4038C000029222002B4F74333B602B4B75321A6022002A4B76321A602300294A77331360220005002000274B783201911A600E300422029900F030FA0396214E012D06D9B6
:403900002000029912300431042200F025FA05AA01992800FFF76EFE059A01992800FFF75BFCFFF735FE002807D1230073331B78AB4202D02800FFF7ABFF002D0FD1230063
:4039400073331B78002B0AD03B680234E577002B00D01D703368002B01D000221A70039B1B68002B00D01D7007B0F0BDEC010020F0030020E4030020B0030020B803002027
:40398000C8030020A40300200100562210B5184800F0E2F90021174A174B126859628A4200D01170154A1268002A01D000211170134A11680022914200D00A701149DA6196
:4039C0000A60114A1268002A01D0002111700F4A11680022914200D00A700D491A600A70991CCA77190049310A701A7110BDC046A8000020F0030020EC010020E403002040
:403A0000C8030020D4030020A4030020B8030020C6030020002243088B4274D303098B425FD3030A8B4244D3030B8B4228D3030C8B420DD3FF22090212BA030C8B4202D361
:403A40001212090265D0030B8B4219D300E0090AC30B8B4201D3CB03C01A5241830B8B4201D38B03C01A5241430B8B4201D34B03C01A5241030B8B4201D30B03C01A524180
:403A8000C30A8B4201D3CB02C01A5241830A8B4201D38B02C01A5241430A8B4201D34B02C01A5241030A8B4201D30B02C01A5241CDD2C3098B4201D3CB01C01A5241830995
:403AC0008B4201D38B01C01A524143098B4201D34B01C01A524103098B4201D30B01C01A5241C3088B4201D3CB00C01A524183088B4201D38B00C01A524143088B4201D3AC
:403B00004B00C01A5241411A00D20146524110467047FFE701B5002000F0F0F802BDC0460029F7D076E7704703460B437FD4002243088B4274D303098B425FD3030A8B420C
:403B400044D3030B8B4228D3030C8B420DD3FF22090212BA030C8B4202D31212090265D0030B8B4219D300E0090AC30B8B4201D3CB03C01A5241830B8B4201D38B03C01A94
:403B80005241430B8B4201D34B03C01A5241030B8B4201D30B03C01A5241C30A8B4201D3CB02C01A5241830A8B4201D38B02C01A5241430A8B4201D34B02C01A5241030A19
:403BC0008B4201D30B02C01A5241CDD2C3098B4201D3CB01C01A524183098B4201D38B01C01A524143098B4201D34B01C01A524103098B4201D30B01C01A5241C3088B42DB
:403C000001D3CB00C01A524183088B4201D38B00C01A524143088B4201D34B00C01A5241411A00D201465241104670475DE0CA0F00D04942031000D34042534000229C462C
:403C400003098B422DD3030A8B4212D3FC22890112BA030A8B420CD3890192118B4208D3890192118B4204D389013AD0921100E08909C3098B4201D3CB01C01A52418309FE
:403C80008B4201D38B01C01A524143098B4201D34B01C01A524103098B4201D30B01C01A5241C3088B4201D3CB00C01A524183088B4201D38B00C01A5241D9D243088B4213
:403CC00001D34B00C01A5241411A00D20146634652415B10104601D34042002B00D54942704763465B1000D3404201B5002000F005F802BD0029F8D016E770477047C046E2
:403D0000014B18687047C046640100200E4B70B500251E000D4CE41AA410A54204D0AB00F35898470135F8E700F098F9084B00251E00084CE41AA410A54204D0AB00F35836
:403D400098470135F8E770BD68400000684000006840000070400000002310B59A4203D0CC5CC4540133F9E710BD03008218934202D019700133FAE7704700000000000029
:403D80009C0300005C02000014030000640300008C020000DA0200002020202020202020D43E0000A0020020DA02002000000000A001002009280000010001020101000056
:403DC00000000000000000000C3F0000AE020020E4020020000000009C0100200128000001000102010100000000000000000000443F0000BC020020EE0200200000000045
:403E00009801002001280000010001020101000000000000000000007C3F0000CA020020F802002000000000940100200128000005000201050064000019000080000000F1
:403E40004B0096004B4B14021E20500000003200C800646419021E20500000002800C800646419021E20500000000B002800141405031E2004000000FFFF0000560808084A
:403E80000014001414141400000000030507090314181E2800000000030507090305320000320000642D2D05030303030000141E000003000B0000005000D007E803640008
:403EC000E8030A00E8030A00F02829303F4849909F0000000001024008010440000104400401044000000F001000000010040C0000010240080104400001044004010440ED
:403F000000F00000080000000C030900000102400801044000010440040104400000F0002000000014050F000001024008010440000104400401044000F000000800000005
:403F40000C030900000102400801044000010440040104400000000F40000000180612000001024008010440000104400401044000F00000080000000C030900000002401C
:403F80000800044000000440040004400F000000010000000000000000000240080004400000044004000440F0000000020000000401030000000240080004400000044033
:403FC00004000440000F000004000000080206000000024008000440000004400400044000F00000080000000C030900000002400800044000000440040004400000000F03
:404000004000000018061200E60E0000A60E0000B00E0000BA0E0000CA0E0000D40E0000DE0E00006E13000094130000FE130000AC130000B4130000DA1300000000000090
:40404000EEDBC9B9AA9B8E82766B60564D443B332C241D17100A044300000000F8B5C046F8BC08BC9E46704795010000F1040000F8B5C046F8BC08BC9E4670476D010000A0
:404080009040000080000020E80000009802000000000000010101010100000020000004B1240000010000000000E02EC05D00001800000000366E0156121212122323142F
:4040C000181E2814181E28030507090314181E2814181E2803050709020A323200323200642D2DC80203020A1401321E1E0028004006B00450002003C8001400C80014009E
:40410000C8006400F02829303F4849909F00FF3FFFFF0000000000000000000000000000000000000000000000000000000000000000000057400000000000000000000010
:40414000000000000000000000000000000000000000000000000000000000000000000000000000000000000000000000000000000000000401002000000000000000001A
:4041800000000000000000000000000000000000000000000000000000000000000000000000000000000000000000000000000000000000000000000000000000000000FF
:4041C00000000000000000000000000000000000000000000000000000000000000000000000000000000000000000000000000000000000000000000000000000000000BF
:40420000000000000000000000000000000000000000000000000000000000000000000000000000000000000000000000000000000000000000000000000000000000007E
:40424000000000000000000000000000000000000000000000000000000000000000000000000000000000000000000000000000000000000000000000000000000000003E
:0200000490303A
:020000006AADE7
:0200000490402A
:200000000000000000000000000000000000000000000000000000000000000000000000E0
:0200000490501A
:0C0000000002190111A9000119157C561D
:0200000490600A
:0100000001FE
:00000001FF
